:100000000BC018951895189518951895189518956A
:1000100018951895189518958FED8DBFC0ECE4EBE9
:100020004E2EDD275D2EEEE7F0E0A0E6B0E0A895CD
:1000300084B7082E877F84BF88E1992781BD91BD51
:1000400088278D933197E9F766248DEF8ABB8FED72
:1000500087BB80E08BBB80E088BBD99A83E886B9F8
:1000600080E087B980E080936800EEE0F0E0A2E6EF
:1000700091E01ED3009162000E3C08F005C085B7E8
:100080008F7E806385BF8895A3E6E3D280E080936E
:10009000670080E080936100ACE6D9D28091740063
:1000A0008F7780937400D198A4E79C9196FF04C049
:1000B000C99B0EC09F7B9C93C9990AC084E69F93FD
:1000C000992774D19F91C99903C090649C930AD1D8
:1000D000AEE6BDD2379A81E080936B0000916B0051
:1000E0000A3010F009F020C0EF93FF93E5E1F0E053
:1000F00054D1FF91EF9107B1007E086007B965D137
:10010000ACE68D939C93AEE60D911C91ACE64D91BF
:100110005C91040F151FAEE60D931C93ABE68C911A
:100120008F5F8C9308F4DACF3798ECE6F0E0D1904B
:10013000E080FF240027B4D1A0E7E3D1EEEDF6E0A4
:100140007DD2E0E7F0E088D1EED1EDE0A0E791D2FA
:10015000E2EEF6E073D2E0E7F0E07ED11DD2EDE012
:100160003DD1A0E6DC92A0E60C914AE0A8D20C9327
:1001700000916000003010F009F001C001C02CD0E7
:1001800084E690E013D100916700063009F022C0A8
:10019000A4E78C9187FB0EF00DC0EAE0F0E0A3E647
:1001A00094E07BE774D25FD0809174008F77809366
:1001B00074005BCFEAE0F0E0A4E194E079D2A3E63A
:1001C0000D911D912D913C914FD209F002C072C04A
:1001D00001C02EC068CF46CFD89A84E690E0E6D022
:1001E000D89884E690E0E2D0A7E68C918F5F8C935C
:1001F000A3E60D911D912D913C914AE050E060E005
:1002000070E085D0A3E60D931D932D933D93A3E657
:100210000D911D912D913C91A0E64C91552766279B
:1002200077271DD2A3E60D931D932D933D9308953B
:1002300084E690E0BBD0A8E68C918F5F8C9389E038
:10024000809369008FE580936A0018D00091680060
:10025000033009F007C0ECE3F0E053D080E0809376
:10026000680001D002CF84E690E0A0D082E08093C5
:10027000690088EC80936A0001D0089581E0809342
:100280006B004091690000916B00041710F009F0B9
:1002900010C0D89AAAE68C91992788D0D898AAE657
:1002A0008C91992783D0ABE68C918F5F8C9308F467
:1002B000E8CF0895D8DF8CE291E078D0DA9AE2E0D6
:1002C000F0E01FD0DA98E1E0F0E01BD0809162000E
:1002D000815080936200EEE0F0E0A2E691E07BE7DF
:1002E000D6D1C3CED89A84E690E060D0D89884E680
:1002F00090E05CD080917400806880937400B3DFDC
:10030000089588EE93E052D03197D9F7089522D01E
:1003100006D000FC01D0089528D030D00895842F55
:10032000952FA62FB72F4427552766277727F1E269
:10033000889409C020F4480F591F6A1F7B1F7695C7
:100340006795579547953795279517950795FA958A
:1003500089F708950024E89477FF02C006D06894D6
:1003600000F809D010F80124089512D04F5F5F4FB4
:100370006F4F7F4F0895E89437FF089500951095CB
:10038000209530950F5F1F4F2F4F3F4F6894089572
:10039000409550956095709508953197F1F70895BF
:1003A000689462F80895E89462F80895EF93FF93D3
:1003B000EE27E82BE92B31F0EAEFF0E03197F1F787
:1003C0000197D1F7FF91EF910895369A3699FECFB4
:1003D000369A3699FECF84B195B108953DD09927CC
:1003E00011278F2D880F80E8F82A802F881F08F4A6
:1003F0001FEF41F08F57082F07FD04C0003240F077
:100400008FEF01C08827982FD82EE82EF82E09C02C
:100410008FE1801B082FF694E794D79497950A955F
:10042000D1F7112351F09095D094E094F09481E0AD
:10043000980F8827D81EE81EF81E0F2DFE2CED2CD5
:10044000D92E0895D094E094F09491E0D90E992794
:10045000E91EF91E10950895D190E190F190019157
:10046000089521913191419151910895102F90E873
:10047000FF0C001F0927990FF7941078652F90E85B
:10048000440F551F5927990F4795607800380895F4
:10049000FF0C90E89027110F9795F794092F089576
:1004A000102FBD2CDE2CEF2CF02E11234AF4B0942B
:1004B000D094E094F0949FEFB91AD90AE90AF90AA6
:1004C0000EE1FF2039F4FE2CED2CDB2CBB24085070
:1004D000C2F723C032F00A95BB0CDD1CEE1CFF1CDA
:1004E000F9CF01D0D5CFB7FE089590E8B91611F431
:1004F000D0FE08959FEFD91AE90AF90A09F4039585
:100500000895DD92ED92FD920C9308959FE7092FD7
:10051000F92A9FEFD92EE92E0895DD24EE24FF2439
:10052000002711270895A2DFC1F35038B1F3162731
:10053000005850580894051F12F418F4E7CF08F03B
:10054000ECCF0AD0FF202AF0BB0CDD1CEE1CFF1CF8
:100550009FCF0F5FDBF29CCF9F929924AA24BB24EC
:10056000992788E1990CAA1CBB1CDD1CEE1CFF1C02
:1005700030F4920EA31EB41ED91EE91EF91E8A95F0
:1005800089F79F9008950AF045D082CF5FE3222734
:100590003327442701C065DF69DF5038B1F30038E5
:1005A00099F3902F951B8BF312F434D0FACF983136
:1005B00018F0222733274427983028F0232F342F90
:1005C00044279850F9CF992329F0469537952795D8
:1005D0009A95D9F7912F962742F014D0B0F6F79458
:1005E000E794D7940F5F8BF691CF10D051F008F4B9
:1005F00029DFFF2052F2DD0CEE1CFF1C0150CBF76F
:1006000085CF8BCFD20EE31EF41E0895D21AE30AD3
:10061000F40A0895DF92EF92FF920F931F93D22E68
:10062000E32EF42E052F162F6F915F914F913F917E
:100630002F910895C895319600200895FBDF202D55
:10064000F9DF302DF7DF402DF5DF502D089582E0E2
:1006500001C084E099279D938A95E9F70895040FD6
:10066000151F261F371F089504171507260737077C
:10067000089594E081918D939A95E1F70895E19919
:10068000FECFEEBB3196089591E001C092E07B373A
:1006900051F47FB7F894F3DF8D918DBBE29AE19A24
:1006A0009A95C9F77FBF7727089591E001C092E03E
:1006B000E6DFE09A8DB38D939A95D1F70895FF9375
:1006C000881BF9E0001FFA9511F4FF910895881F27
:1006D000841B18F4840F8894F5CF0894F3CF00009E
:0606E000003E0000004096
:00000001FF
